:100000000C942A000C9445000C9445000C94450077
:100010000C9445000C9445000C9445000C9445004C
:100020000C9445000C9445000C9445000C9445003C
:100030000C9445000C9445000C9445000C9445002C
:100040000C9445000C9445000C9445000C9445001C
:100050000C94450011241FBECFE5D8E0DEBFCDBF14
:1000600010E0A0E6B0E0E6EDF1E002C005900D92F0
:10007000A036B107D9F710E0A0E6B0E001C01D92AC
:10008000A036B107E1F70C94DB000C94000084E883
:1000900086B908951CBE13BC89E683BF85BD08954B
:1000A000882321F4662341F4C09A0895662311F44D
:1000B000C19A0895C1980895C09808950895882315
:1000C00011F46CBF0895813009F0089563BD08955F
:1000D0000895877087B9369A3699FECF84B195B165
:1000E00008950F931F93CF93DF9380E00E946900E0
:1000F00097FD46C0EC01D595C79581E00E94690047
:1001000097FD47C0BC0175956795CF5FD0406F5F85
:100110007040CE010F964F9710F4C0E0D0E0CB01B5
:100120000F964F9710F460E070E08E01060F171FD6
:100130006C1B7D0BEB0117FD36C061E080E00E9477
:100140005000D7FD28C061E0862F0E9450000F3F6D
:10015000110519F014F00FEF10E0CF3FD10519F0A1
:1001600014F0CFEFD0E0602F80E00E945F006C2F92
:1001700081E00E945F0080E00E94690097FFBACF93
:100180000196EC01D595C79581E00E94690097FF23
:10019000B9CF0196B7CF60E081E00E945000D095C2
:1001A000C195DF4FD4CF60E0862F0E94500010959C
:1001B00001951F4FC6CFCFE5D8E0DEBFCDBF8FEF93
:1001C00087BB81BB0E9447000E944A000E947100C9
:0601D0000C94EA00FFCFD1
:00000001FF
